:020000020000FC
:1000000012C0189518951895189532C0189518951E
:100010001895189518951895189518951895189578
:100020001895189518950FE50DBF04E00EBF20E355
:1000300037E310E060E070E00FE004BB09B7006256
:1000400009BF02E40EBD0CE009B900E000BD06E8FE
:1000500000BD539A789410FFF1F7092F1AD0082F9A
:1000600018D017FF02C032D001C02BD010E0F3CF60
:10007000FFB646B557B5CA01861B970BBA0111E00A
:10008000933128F060E070E06DBD6CBD1FEFFFBEE6
:100090001895E02E06950695069506950A3014F4F7
:1000A000020F01C0030F5D9BFECF0CB90E2D0F7028
:1000B0000A3014F4020F01C0030F5D9BFECF0CB990
:1000C00008950CE25D9BFECF0CB908950AE05D9B9C
:0E00D000FECF0CB90DE05D9BFECF0CB908957C
:00000001FF
